:020000040001F9
:10B00000A83F002039B1010053B1010055B1010042
:10B010000000000000000000000000000000000030
:10B0200000000000000000000000000057B1010017
:10B03000000000000000000059B101005BB10100F8
:10B040005DB101005DB1010035BC01005DB10100E1
:10B05000D1BA010000000000EDB701005DB10100B0
:10B060005DB101005DB101005DB101005DB10100A4
:10B070005DB101005DB101005DB101005DB1010094
:10B080003DBC0100B1BA01005DB101005DB101003C
:10B09000E5BA01005DB10100EDBA01005DB101004A
:10B0A0005DB101005DB10100000000000000000082
:10B0B0000000000000000000000000000000000090
:10B0C0000448854600F0C2FA0048004795E60100B2
:10B0D000C046C046A83F0020401E00BF00BF00BFC2
:10B0E00000BF00BF00BF00BF00BF00BF00BF00BF68
:10B0F00000BFF1D170470000401E00BF00BF00BF7D
:10B1000000BF00BF00BF00BF00BF00BF00BF00BF47
:10B1100000BFF1D170470000401E00BF00BF00BF5C
:10B1200000BF00BF00BF00BF00BF00BF00BF00BF27
:10B1300000BFF1D1704700000321094802680A43AB
:10B140000260084802680A430260074880470748CF
:10B150000047FEE7FEE7FEE7FEE7FEE7FEE700004A
:10B16000240500405405004095BB0100C1B001001A
:10B1700030B50B46014600202022012409E00D468F
:10B18000D5409D4205D31D469540491B2546954017
:10B1900040191546521E002DF1DC30BD70B500245B
:10B1A0002546002801DA01244042002901DA012560
:10B1B0004942FFF7DDFFAC4200D04042002C00D0F6
:10B1C000494270BD03460B439B0703D009E008C901
:10B1D000121F08C0042AFAD203E00B780370401C47
:10B1E000491C521EF9D27047D2B201E00270401CD5
:10B1F000491EFBD270470022F6E710B513460A46F7
:10B2000004461946FFF7F0FF204610BD421C0178A6
:10B21000401C0029FBD1801A704730B5044600203D
:10B22000034600E05B1C934203D2E05CCD5C401B14
:10B23000F8D030BD03460A780270401C491C002A31
:10B24000F9D1184670470022CBB20178994200D15B
:10B250000246401C0029F8D110467047F0B51FB4D3
:10B260000646002082B005464024019100901BE074
:10B27000019922460F46304600F00AFA049A059BCF
:10B28000801A994110D310461946224600F0F0F971
:10B29000361A8F410197224601200021009F00F0BD
:10B2A000E7F938184D4100902046641E0028DFDC85
:10B2B000019B00982946324607B0F0BDF0B507461D
:10B2C0000846584087B0C00F049048000E46590009
:10B2D00040084908BC1A884105D2384631461E4606
:10B2E00017460B4602465800400810434DD0300D1B
:10B2F000039040055900400D490D0590401A0290F9
:10B30000402873DA18030121000B09050843019056
:10B3100004980092002806D01146019A4942002064
:10B32000904100910190029840210A1A01990098D9
:10B3300000F09EF905460C466B4607CB00F0B9F9C4
:10B34000C0197141039A0E0D0023D71756401A46B3
:10B350007A40164344D0049A002A2DD0029A012A3A
:10B36000039A15DC1205C01A914101263605001C0E
:10B370007141D20F059ED2070093019202962A4690
:10B38000234600F0B6F907B0F0BD38463146FAE77B
:10B390001605234A0F46B218C01AB7410121090504
:10B3A000001C4F4100187F41114618187941E20FE7
:10B3B00010436D19644113E0E2076D0815436408FA
:10B3C000C2071443039A01261205C01A914136059B
:10B3D000001C7141CE07400830434908C018514154
:10B3E0002A46234600F078F9CDE7FFE704980122CA
:10B3F0004000C117121A00238B4104983146C4172C
:10B40000381AA141EEE730B40124E407634030BCB0
:10B4100054E730B40124E407614030BC4EE700003B
:10B420000000E0FFF0B51FB488B00B990998002424
:10B4300048400999C00F490049080991C0070B9974
:10B440000090490049080B9109990898A6460843BD
:10B450001CD00B990A98084318D009980124400081
:10B46000420D4800410D099824050003000B2043BC
:10B4700009900B980003000B20430B9050181C49B7
:10B480004018002201901446104605E000200146B5
:10B490000DB0F0BD032801DA034600E003239C460B
:10B4A000C11A0AAE0AE05F0008ADED5B4F00F75B22
:10B4B0007D430027AA187C41491C5B1E6145F2DDD3
:10B4C000410004AB5A522104120C0A43240C401CC4
:10B4D0000828DFDB019802900099704601910090E6
:10B4E000059B049A0799069800F003F9D0E700003D
:10B4F0000DFCFFFFF0B50C465C4085B0E40FE4079F
:10B5000003944C00002664085900944649080246FA
:10B510000296224321D062460A431ED06200570D94
:10B520004A000E032303550D012402462C4924052D
:10B53000781B1B0B360B40182343264361460090B3
:10B540001C46501AB44103D30098401C009002E0FE
:10B55000921800985B41002803DA0020014605B0EC
:10B56000F0BD0020012109050746864611E064462A
:10B570001D46141BB54106D36546521BB3417446A4
:10B5800007430C43A646CD074008490828439218B4
:10B590005B4105460D43EAD11046184313D060467F
:10B5A000194650407140084306D06046101AB34116
:10B5B00006D20122002306E000220123DB0702E07D
:10B5C0000122D2435310009874460105381C614192
:10B5D000029C039D0019694100F07EF8BFE700005E
:10B5E000FD0300004A0009030123090B1B05194351
:10B5F0000A4B10B5520D9A4202DA0020014610BDE6
:10B60000064B34339A4203DC9A1A00F041F810BD1D
:10B61000034BD21800F02CF810BD0000FF0300000F
:10B62000CDFBFFFF10B5002904DB0124E4074042F5
:10B630008C412146002B04DB1C460123DB075242D0
:10B64000A341994200D1904210BD0000064C012553
:10B65000064E05E0E36807CC2B430C3C98471034BA
:10B66000B442F7D3FFF730FDCC0C0200EC0C020023
:10B6700010B5202A04DB0146203A9140002010BD7D
:10B68000914020239C1A0346E3401943904010BD8B
:10B6900010B5202A04DB0846203AD040002110BD16
:10B6A0000B46D340D0402024A21A914008431946AB
:10B6B00010BD10B5202A06DBCB170846203A1041F2
:10B6C000C1170B4306E00B461341D0402024A21AB9
:10B6D00091400843194610BD10B5002B08DA00242C
:10B6E000401C614192185B411A4301D1400840005F
:10B6F00010BDF0B51FB482B005460C0003D008465B
:10B7000000F0CEFA02E000F0CBFA203002460090C2
:10B7100021462846FFF7ACFF049B059A04460F46D6
:10B7200018431143084314D0184610431BD0009807
:10B7300040210A1A18460599FFF7AAFF05460E464A
:10B74000009A05990498FFF793FF084305D001205C
:10B7500004E02046394607B0F0BD0020C11705437C
:10B760000E432C43374300990E986305401A790520
:10B77000E40A00220C43FD0A0A3002D500200146EB
:10B78000E9E70105101969410C9C0D9D00196941FB
:10B79000FFF7A2FFDFE770B58C180578401C6B0738
:10B7A0005B0F01D10378401C2A1106D10278401C9E
:10B7B00003E006780E70401C491C5B1EF9D12B0774
:10B7C00005D40023521E0DD40B70491CFAE70378F0
:10B7D000401CCB1A921C03E01D780D70491C5B1CA9
:10B7E000521EF9D5A142D8D3002070BDF0B5002576
:10B7F000FF248BB0013401262F460195204603F02B
:10B8000037FC002808D047484068304204D04648FA
:10B810000021201835430160241D76007F1CA4B24E
:10B82000042FEBD3FF207D3003F022FC002807D04B
:10B830003E4800210160400705433D4800690190F2
:10B840003C4C280712D0012700262F420AD03A4844
:10B85000B200111808690969C004C00E8903A25812
:10B86000890F90477F00761C042EEED3002D57DA07
:10B8700000200590401E4DE0A11940310878850652
:10B88000AD0E42B2521C39D00121A940089A009154
:10B89000114233D080090390284601F0D7FF800081
:10B8A00020580490002802D10398032826D1039839
:10B8B0000099032802D10598084305901F4AA80063
:10B8C00080180068019A8003800F114202D002287C
:10B8D00002D013E0032811D10399032907D10228CC
:10B8E0001CD00221284603F0B3FB7F1CFFB2049852
:10B8F000002803D0049A284603999047761C042E0A
:10B90000BAD3002F0CD00A4800690199884207D0A9
:10B910000190059800273E460890ADE70321E1E736
:10B920000BB0F0BD00630040006000407C6100404F
:10B9300000050050202F0020006500400007005047
:10B94000F3B581B00746002414210298FFF710FCDC
:10B95000064630480D4680882F49884219D15C211F
:10B960002EA0FFF770FC002805D05C212BA0FFF76C
:10B970006AFC401C00E029A0FF22014674322BA083
:10B9800002F07EFE2CA002F07BFE30A002F078FEDA
:10B99000FEBD5C2121A0FFF756FC002805D05C21EC
:10B9A0001EA0FFF750FC401C00E01CA0FF22014637
:10B9B00077321EA002F064FE3846029900F0A6F825
:10B9C000014623A0029A02F05BFE20A002F058FE7E
:10B9D0000EE014206043C1191422234801F0BEFE7A
:10B9E000641CE4B2082803D0002801D000F0C2FF94
:10B9F000B442EED3002DCBD014204443E1192A46A3
:10BA0000194801F0ABFE0828C2D00028C0D000F0D1
:10BA1000B1FFFEBD80200020FFFF00002E2E5C2E17
:10BA20002E5C2E2E5C6D61696E2E63005B25735D4E
:10BA30005B25645D3A000000626C65206469736395
:10BA40006F6E6E6563746564000000000D0A00008F
:10BA5000626C655F74785F646174613A25732C6C05
:10BA6000656E3A2564000000382600208307FF2217
:10BA7000DB0E9A408907090E994000280BDA00076F
:10BA8000000F0838830808489B001818C3699343BF
:10BA90000B43C3617047830804489B001B18186858
:10BAA000904308431860704700ED00E000E400E0B8
:10BAB00010B506490020086048608860C8600349E6
:10BAC00040390860486004F06BFD10BD4011014032
:10BAD00010B50249024804F0B5F910BD68300020E5
:10BAE0000040004010B504F0B3FC10BD10B506488E
:10BAF0004068002805D08047002801D000F03AFFB8
:10BB000010BD02F0DFFB10BDBC210020FEB50325F7
:10BB10002D020646A94200DC0D460E490E48FFF7ED
:10BB20006AFB00240C4F0DE0325D0CA1684600F06A
:10BB300099F86000C1196846007808706846407836
:10BB40004870641CAC42EFDB0649002008700248D4
:10BB5000FEBD00000106000064330020253032588D
:10BB6000000000006439002070B50D460646002430
:10BB700004E0315D04A002F083FD641CAC42F8D304
:10BB800003A002F07DFD70BD25303258000000009A
:10BB90000A00000010B502F0DFFB002805D01F49A5
:10BBA0001D484860C8131E4988611E48018CC9B2EF
:10BBB00001290BD1828C120708D1028D1206120FB7
:10BBC000042A03D1828D1206120F0AD0012921D135
:10BBD000818C09071ED1018D0906090F0A2904D09D
:10BBE00007E0114A01219160F5E7828D1206120FDC
:10BBF00005D00D290ED1808D0006000F0AD10B480B
:10BC00000168012904D00A49016001680129FCD1B9
:10BC1000C021416110BD0000DFFF07C000050040EA
:10BC2000006C0040C00F00F00006004000EC064031
:10BC30007593000010B504F0E3FD10BD06484068A0
:10BC4000C107C90F0020002904D004490860044836
:10BC500040680047704700000003014000010140B8
:10BC6000B02100200FB410B504A9074B02AA039815
:10BC700000F0F6F8044602A9002000F08FFC2046F0
:10BC800010BC08BC04B018479DC5010010B5024B9C
:10BC9000024A00F0E5F810BD61E10100F821002042
:10BCA0002021020C01D010211046020A01D01046BA
:10BCB0000839020901D01046091F820801D0104638
:10BCC000891E420801D0881E7047081A704702E09A
:10BCD00008C8121F08C1002AFAD170477047002017
:10BCE00001E001C1121F002AFBD17047F0B51FB45B
:10BCF00086B00998089A030D0021024314D05148D8
:10BD0000514A1818504305141198012810981AD058
:10BD1000281A401C00264D4F4D4900960191049071
:10BD2000002812DA444211E01198012449A30128A5
:10BD300001D11098C1430698119A84600360C260D3
:10BD400041600BB0F0BD4042E4E70446210500200D
:10BD50003F4A001C51410391029012E0E00707D0D6
:10BD600032463B4601990098FFF75CFB0191009039
:10BD700032463B4610461946FFF754FB06460F462F
:10BD80006410002CEAD10498039B0028029A0999B8
:10BD9000089806DAFFF746FB019B009AFFF742FB83
:10BDA00005E0FFF7A7FB019B009AFFF7A3FB044602
:10BDB0000E460022284BFFF735FC03D80020C04375
:10BDC000014607E00022254B20463146FFF776FA70
:10BDD000FFF708FC102409E0002C0ADB0A220023EC
:10BDE000FFF73CFA079B30321A55641E02460A439D
:10BDF000F2D11122641C079B121B1C19119B012BF1
:10BE000003D0012308430ED10AE0084304D01120D7
:10BE100010900020119077E71098151A6D1E0BE016
:10BE20001098824202DD00236D1C03E0824201DA99
:10BE300000236D1E002BEED0069811998260C16020
:10BE400030C07EE701FCFFFF104D000000001440F1
:10BE50000000F03F300000000000F0430000E03F31
:10BE6000FFB597B0064600251BE2252876D10024B1
:10BE70002746F749049400E00443761C32780120F9
:10BE8000203A90400842F7D130782A280ED002227A
:10BE9000307801463039092916D804990A235943C4
:10BEA000303940181443761C0490F1E7189802C802
:10BEB00004911890002904DA012040030443484209
:10BEC000049002200443761C30782E2814D10420DC
:10BED00004437078761C2A2809D11898761C80C8EB
:10BEE000189009E00A214F43303FC719761C30787B
:10BEF000014630390929F5D930786C2810D006DC94
:10BF00004C281AD068280ED06A2817D104E074286B
:10BF100013D07A2812D110E00120400504430CE030
:10BF20000121090501E0032109050C4371788142D3
:10BF300003D1012000052418761C761C3078662871
:10BF40000BD013DC58287DD009DC00287BD0452895
:10BF5000F6D04628F4D047281AD1A9E118E0632882
:10BF600035D0642870D0652812D1A1E170286CD03A
:10BF700008DC6728F1D069287DD06E280DD06F28A5
:10BF800006D1BCE073282ED0752873D0782859D0FC
:10BF90001A9A199990476D1C82E16002400F02289D
:10BFA00009D003280DD00428189801680DD00D6021
:10BFB000001D189074E11898EA1701680D604A6036
:10BFC000F6E7189801680D80F2E70D70F0E7189811
:10BFD0006A4601781172001D18900020507202A864
:10BFE0000090012005E0189802C8189000200091E8
:10BFF000C04361070ED5002101E00199491C019160
:10C00000B94213DA8142F8DB019A0099895C002970
:10C01000F3D10BE0002101E00199491C019181421B
:10C02000FADB019A0099895C0029F5D101990498FD
:10C030001A9B471A21463846199A00F099FA401976
:10C04000019903E051E030E115E050E0451807E0C8
:10C05000009800990078491C00911A9A1999904704
:10C060000198401E0190401CF2D1214638461A9B8F
:10C07000199A12E137E00A20002100900191600234
:10C08000410F022907D0189A01CA1892C217944684
:10C09000032908D00AE01898C01DC108C90005C9C5
:10C0A0001891944607E000B2C2179446042902D1C1
:10C0B00040B2C1178C4600226146944506DA0A4612
:10C0C0000021404291418C462D2102E0210504D5FA
:10C0D0002B216A461173012103E0E10701D02021E1
:10C0E000F7E7029156E00A200AE0102008E010204D
:10C0F00000900021042004430191082703E0082058
:10C100000021019100906002410F022907D0189A86
:10C1100001CA189200229446032908D008E0189812
:10C12000C01DC108C90005C91891944603E080B23A
:10C13000042900D1C0B20021029121072AD531780B
:10C140000D91702906D0009A1021019B4A401A4394
:10C1500005D00EE040216A461173012108E06146D6
:10C16000014306D030216A4611730D9951730221A3
:10C170000291009A0821019B4A401A430AD1614664
:10C18000014301D1610705D530216A4611730121B0
:10C190007F1E02913178582904D02EA10E910DA94D
:10C1A0000D910DE030A1F9E76146019B009AFFF780
:10C1B00055F80E9B8C469B5C0D9A521E0D92137087
:10C1C00061460143F0D10D9805A9081A203001906D
:10C1D000600703D501200004844300E00127019893
:10C1E000874201DD381A00E00020019900904118D3
:10C1F000029809180498401A0490E00306D42146D6
:10C200001A9B199A049800F0B3F94519002706E023
:10C2100003A81A9AC05D199990476D1C7F1C02985B
:10C220008742F5DBE0030CD521461A9B199A049846
:10C2300000F09EF9451904E01A9A302019999047A8
:10C240006D1C0099481E00900029F5DC1FE00000DD
:10C2500009280100303132333435363738396162DC
:10C2600063646566000000003031323334353637A0
:10C270003839414243444546000000000D980D996D
:10C280000078491C0D911A9A199990476D1C0199D3
:10C29000481E01900029F1DC4DE100F059F94519E3
:10C2A000761C3078002800D0DFE528461BB0F0BDB2
:10C2B000600700D406271898C01DC108C900486847
:10C2C0000A680831C30FDB071891190001D09CA13F
:10C2D00008E0210501D59BA104E0E10701D09AA166
:10C2E00000E09AA14300109130785B0865280CD0DB
:10C2F00006DC452809D046281DD0472841D141E019
:10C30000662818D067283CD13CE00021112F01DBC2
:10C31000112000E0781C0191009008A911A8FFF7F6
:10C32000E5FC139905910021119A15927F1C129832
:10C330000197009150E00120C00703900120019077
:10C3400008A9009711A8FFF7D1FC139A1499059238
:10C350000022119B009212981593059A01920029D0
:10C3600001D0104602E0791C40180190381A01D51E
:10C37000019804E04042401E0090781C0190C01BD0
:10C38000029043E0012F00DA01270021112F01DD87
:10C39000112000E038460191009008A911A8FFF78C
:10C3A000A5FC13990591119A0021129815920091FC
:10C3B000019721070CD40599B94201DB019900E0EE
:10C3C0000191012904DD159A491E515C302906D0DE
:10C3D000B84201DA011D05DA0121029115E0019947
:10C3E000491EEDE7002805DC0099411800910199EC
:10C3F000091A03E0019A411C914200DD0191009964
:10C40000401A401C02900120C0070390200706D468
:10C4100002990198814202DB0020C0430290002073
:10C420006946C87707AF012103980337C9078842D7
:10C4300024D0022011902B201290039800280CDAAF
:10C44000404203902D20129007E00A210398FEF746
:10C450008FFE30317F1E039039701199481E119064
:10C460000029F2DC03980028EFD1791E1298087099
:10C470003078202108404530BF1E387006A8C01B08
:10C48000C01D039010980078002800D00120019969
:10C4900041180298C0170918039809180498401AFF
:10C4A000401E0490E00306D421461A9B199A049872
:10C4B00000F05EF8451910980078002803D01A9A09
:10C4C000199990476D1CE00324D521461A9B199AAF
:10C4D000049800F04DF845191CE00098002807DB8F
:10C4E00000990598884203DD1598405C199901E090
:10C4F000199930201A9A904700986D1C401C0090A2
:10C500000298401E0290002804D11A9A2E201999F0
:10C5100090476D1C0199481E01900029DDDC05E063
:10C5200038781A9A7F1C199990476D1C0399481EF8
:10C5300003900029F4DC21461A9B199A0498ACE672
:10C540002D0000002B000000200000000000000073
:10C55000F8B5044600251E461746880404D405E0B5
:10C5600039462020B0476D1C641EF9D52846F8BD19
:10C57000FFB50446002581B01E46C80301D530270B
:10C5800000E02027880404D505E038460399B04729
:10C590006D1C641EF9D5284605B0F0BD0A68531C11
:10C5A0000B6010707047000010B57D20C000FEF7D2
:10C5B00093FD04494868401E486001D0002010BD2A
:10C5C000012010BDCC200020F7B584B000251688CE
:10C5D00007461580406B1446002813D00378059851
:10C5E000032E51D30221017021881122491C89B2E6
:10C5F000218042542188491C89B2218043542088DB
:10C60000401C2080386B00281DD0054620880599E5
:10C6100002461232B24237D811220A542088102220
:10C62000401C80B220800A542088401C20800F20AB
:10C630002A5C2388401ECA54228840B2521C2280A1
:10C640000028F5DA0025384620300290807B00284B
:10C6500006D033462246059901F0CAFE050014D1E2
:10C660000298407B002806D032462146059800F00B
:10C670007BFF050009D1B878002823D005988646AD
:10C680002088001DB04202D90C2007B0F0BD6846DA
:10C6900079DF0028F9D12188032072465054208880
:10C6A0001921401C80B22080115420887146401C02
:10C6B00080B2208041186846008804F035F921884E
:10C6C00040182080F878002817D0218803230A46D4
:10C6D000FB56C91C0598B142D6D802218154218845
:10C6E0000122491C89B2218042542188491C89B207
:10C6F000218043542088401C20807868002817D06F
:10C7000021880023C3560A46C91C0598B142BBD8EC
:10C710000221815421880A22491C89B22180425475
:10C720002188491C89B2218043542088401C2080E4
:10C73000388900280AD00094384601960622022142
:10C740000830059B04F081F905009ED1388A002845
:10C750000AD0009438460196072203211030059B29
:10C7600004F073F9050090D1388B00280AD00094AA
:10C7700038460196152214211830059B04F065F9FE
:10C78000050082D1386A002806D033462246059932
:10C7900001F0E6F90500D8D1786A002806D03346C2
:10C7A0002246059902F0DCF80500CED10298007B04
:10C7B000002807D0334622463846059903F0DCF9B5
:10C7C0000500C2D13878002807D0334622463846C3
:10C7D000059902F0F9F80500B7D1284655E70000A1
:10C7E00030B54149ABB0486C896C2A91299013212E
:10C7F00020A8018329A82890062520A88583382110
:10C8000001A8FEF7F8FC022168460171002484713A
:10C81000C57126A80A9038210FA8FEF7ECFC012567
:10C8200010A8858130482421083014901DA8FEF7F7
:10C83000E2FC20A805702C4D5C21E8882190229410
:10C840002AA0FEF700FD002805D05C2127A0FEF7F6
:10C85000FAFC401C00E025A0FF2201465D3227A023
:10C8600001F00EFFE98828A001F00AFF2CA001F0DA
:10C8700007FF2C4B1DAA0FA901A8009400F0DCFAB9
:10C8800000280DD000F076F85C2118A0FEF7DBFC44
:10C8900000281AD05C2115A0FEF7D5FC401C15E03D
:10C8A0005C2112A0FEF7CFFC002805D05C210FA070
:10C8B000FEF7C9FC401C00E00CA0FF2201466332D9
:10C8C0000EA001F0DDFE18A007E008A0FF2201463F
:10C8D00067320AA001F0D4FE19A001F0D1FE10A029
:10C8E00001F0CEFE2BB030BD802000202E2E5C2E1D
:10C8F0002E5C2E2E5C6D61696E2E63005B25735D70
:10C900005B25645D3A00000073657420626C6520ED
:10C9100061647620696E74657276616C3A25640094
:10C920000D0A000031F10100626C652061647665DA
:10C9300072746973696E67207375636365737300DE
:10C94000626C65206164766572746973696E6720D4
:10C950006661696C00000000BFF34F8F0449034813
:10C96000C860BFF34F8F00BFFDE700000400FA0569
:10C9700000ED00E00EB50021029000916A460191A1
:10C980000148FFF7E9FF0EBD0140000010B58268C5
:10C99000C368934203D001F075FB002010BD052051
:10C9A00010BD002906D0002A02D0531E134203D026
:10C9B000092070470E20704701608380002181604C
:10C9C000C1600846704710B58268C3689A1A8388A8
:10C9D0009A4203D801F060FB002010BD042010BD76
:10C9E000F8B50C460E78896803290DD00C22514306
:10C9F000074A555807490246096A009120463146C0
:10CA000008302369A847F8BD024924310D68F1E7D1
:10CA1000503000208821002010B5064914230A78E0
:10CA20005A435118091DFFF7DBFF042003F0ECF80F
:10CA300010BD0000842F00200A4B9B68002B07D0FC
:10CA4000002A07D0002805D00068037C002B03D003
:10CA50000820704707207047002303744174426127
:10CA600018467047D8210020FFB59007002581B0F7
:10CA700014460E46002832D11B4F002C31D002F054
:10CA800079FF0498786103203870334618212246D4
:10CA900000204B43BC601834C10089180D704D70E4
:10CAA0008E704C601C19401C0328F5DBFD607D7006
:10CAB00001240E48BD702405046003211420FEF7F4
:10CAC000D5FF0B4804600B4C0198A0600321112096
:10CAD000FEF7CCFF60683861002005B0F0BD07208C
:10CAE000FBE7BD60FBE70000D821002080E200E00A
:10CAF00000E100E000150140FEB50D461B49174658
:10CB00008968044600292AD0002C28D0052D01D29E
:10CB10000720FEBD6069002821D0607C012820D05C
:10CB2000002603F055FFC0001049019089684018A5
:10CB3000694603F077FF002815D0012101700C49E8
:10CB4000446049680830E2C0084901988968411882
:10CB500068460078487003F0BDFC0020FEBD082048
:10CB6000FEBD2E46DDE70420FEBD0000D8210020DA
:10CB700000150140F8B5134D0446A96800291CD0E2
:10CB8000002C1AD06069002817D00026267403F004
:10CB90001FFFC700A8686946381803F043FF002844
:10CBA0000DD0022101704460A868391868460078E9
:10CBB000487003F08FFC3046F8BD0820F8BD042013
:10CBC000F8BD0000D821002070B50446224888B086
:10CBD0001E460D0042601CD0A888296882B21F48FA
:10CBE000FFF7DFFE002815D1A889A96882B21B488B
:10CBF0001030FFF7D6FE00280CD1202218496846D5
:10CC0000FEF7E0FAA06806902079002804D0012100
:10CC100003E0072008B070BD002168460175067763
:10CC20006079002800D00E2069464875E0780290AF
:10CC3000A0780390207801906078009009496846B8
:10CC400002F036F80028E5D102F0BCF802480121D4
:10CC5000401C02F091F8DDE780210020002F002029
:10CC6000340C02005107020010B501460A48FFF7D4
:10CC7000AAFE04000ED102F04BF900280AD10749A0
:10CC80000548FFF783FE002804D10121034802F084
:10CC9000F3F80446204610BD102F0020802100200C
:10CCA00030B5EFF3108172B6094A54680123002CA5
:10CCB00004D00370002900D162B630BD5360054B2B
:10CCC0001D68054C254015601C6000220270F1E7CC
:10CCD000D021002080E100E0FC06FFBC08494A6842
:10CCE000002A0CD000280AD1EFF3108072B60A682F
:10CCF000044B1A6000224A60002800D162B67047D7
:10CD0000D021002000E100E01CB502F07FFB000410
:10CD1000000C10D1012000070069694688800220BC
:10CD2000C8800548009075200449C00248606846E4
:10CD300002F0F2FB80B21CBD99090200E020002045
:10CD4000F8B515460F4A07460E4610460121083829
:10CD500002F018FB0004000C13D10A4C2B46143CC3
:10CD6000A07032460749384602F080FB05042D0CBE
:10CD700003D005E0052001F077FEA0780028F9D067
:10CD80002846F8BDE8200020F8B515460F4A0746AA
:10CD90000E4610460121083802F0F4FA0004000C97
:10CDA00013D10A4C2B46143C607032463946074872
:10CDB00002F036FC05042D0C03D005E0052001F03F
:10CDC00053FE60780028F9D02846F8BDE8200020FE
:10CDD000F0B50C4693B01F216A4611800726002744
:10CDE0009180002809D0C17849070DD502A9FFF725
:10CDF000EBFB002809D102AD01E000251780002CD3
:10CE00000ED0E078002802D0304613B0F0BD01AA61
:10CE10000AA92046FFF7D8FB0028F6D10AAA02E0AB
:10CE200068460022878068468088C3B268460088CA
:10CE3000C1B2284672DFE8E770B50D460499164680
:10CE4000040042D0002E40D0424800224271C3600C
:10CE50000161242231464048FEF7B4F900F0D4F8CD
:10CE60003D49343108461038016020318160382155
:10CE70005C38FEF7C0F93848217838380170A1785D
:10CE80008170E178C17061784170626921694261A5
:10CE90000161E268A168C26081600146E369A2693C
:10CEA000CB618A61616A002919D00146AC31024622
:10CEB000B83241628A60636A1B880B80616A436A88
:10CEC000898899800021436A06E00E2070BD666A59
:10CED000B668765C5654491C9E888E42F7D8A16A83
:10CEE00000291CD01C4AAC3211460C398A60816280
:10CEF000A36A9B888B80A16A836A098819800021B4
:10CF0000836A04E0A66AB668765C5654491C9E881B
:10CF10008E42F7D82C210A5D0F4918390A73216A0D
:10CF2000002909D00B4914310162226A52884A80D3
:10CF3000216A026A098811806168002904D00549C4
:10CF4000891D416061684160034829463838FFF710
:10CF50003FFF70BD4C210020F82D002010B5028845
:10CF60001C4C102A17D00021112A1AD01B2A11D1CB
:10CF7000007A00280ED1607901281ED0022822D024
:10CF8000032822D0042805D12171E2680846002A2E
:10CF900000D0904710BD817D0129FBD18088208180
:10CFA00010BD6170808821898842F9D1012005E097
:10CFB00021690029F4D0884710BD022000F02CF828
:10CFC0000028F5D110BD0320F8E7032020710420CC
:10CFD000F4E700004C21002010B5022801D00328FE
:10CFE0000ED1084C207800280AD0002020706079EB
:10CFF00000F012F8002803D02169002900D08847EA
:10D0000010BD00004C21002010B507210148FEF79B
:10D01000F2F810BD64210020F0B5784C87B0607143
:10D02000002606A8069602F099F90127082802D0E2
:10D03000002808D104E006A801F09AF8002804D1DD
:10D040000698002801D02770D4E0FFF7DDFF6C4D73
:10D050006878002802D06079012807D0A8780028D5
:10D060000CD06079012801D0022824D1E168002980
:10D0700003D0E7700820884700E0E6706079012857
:10D0800008D16878002809D05C48193002F016F9F8
:10D09000002803D06079022802D00CE002206071E1
:10D0A000A878002805D05548193002F007F9002863
:10D0B00001D103206071287B002804D16079032806
:10D0C00001D104206071287E002804D160790428F1
:10D0D00001D166712671E16800290AD060790328C0
:10D0E00001D0042805D12878002802D060780028D3
:10D0F00017D0A67018216846FEF77DF868460670BE
:10D10000019606720396607901280ED0022815D088
:10D110003B4E243637465C3F03281BD004285DD1A4
:10D120003AE0A77007208847E4E7344818300190B8
:10D130006846077046820682277152E02F481830F1
:10D1400001906846077029894182A98801820220DE
:10D15000207146E0A88A69464882288A08822848C1
:10D16000243003F016FD002805D02878002802D0CE
:10D170006078002801D003202FE002206946087261
:10D1800004200396F8701E4800213838FFF720FE6F
:10D19000002830D1052020E0A88B69460882288C21
:10D1A00048821748243003F0F4FC002805D0287882
:10D1B000002802D06078002801D004200DE0022071
:10D1C0006946087204200396F8700D48002138382B
:10D1D000FFF7FEFD00280ED106202071607900289F
:10D1E00003D0684673DF002805D1E168002901D02B
:10D1F00020798847002007B0F0BD00004C210020B6
:10D20000F82D002070B5064688B00D460024604811
:10D2100003F006FA29465FA001F032FA29463046AB
:10D22000FEF7A2FC0020039004900590069003AB4B
:10D230002A463146022002F07DFD05AB2A463146E2
:10D24000012002F077FD5C2158A0FDF7FCFF0028CB
:10D2500005D05C2155A0FDF7F6FF401C00E053A06F
:10D26000FF220146993255A001F00AFA6846427E33
:10D27000017EC07D6B4607C36846837D427D017D8C
:10D2800051A001F0FDF957A001F0FAF95C2147A087
:10D29000FDF7D9FF002805D05C2144A0FDF7D3FF9E
:10D2A000401C00E041A0FF2201469A3243A001F059
:10D2B000E7F903A8FDF7AAFF024603A94AA001F077
:10D2C000DFF948A001F0DCF9314910223B3103A815
:10D2D000FDF7A3FF002811D02C22102103A8FFF78F
:10D2E00053FD010006D046A001F0CAF90020C0435A
:10D2F00008B070BD0124642001F0B6FB07AB2A46DC
:10D300003146032002F016FD05465C2127A0FDF7FB
:10D310009AFF002805D05C2124A0FDF794FF401C53
:10D3200000E022A0FF220146AB3224A001F0A8F9C0
:10D330003DA0079901F0A4F92AA001F0A1F9002D60
:10D3400018D013490422333107A8FDF766FF0028DF
:10D3500010D02422042107A8FFF716FD010005D0F4
:10D3600037A001F08DF90120C043C1E76420641C9F
:10D3700001F07AFB002C08D0BFF34F8F3C493B48AB
:10D38000C860BFF34F8F00BFFDE70020B0E700008B
:10D3900081200020727820626C65206366672C6CA7
:10D3A000656E3A25642C646174613A002E2E5C2E01
:10D3B0002E5C2E2E5C6D61696E2E63005B25735DA5
:10D3C0005B25645D3A000000626C6520636667203F
:10D3D0006D61633A255825582558255825582558F4
:10D3E000000000000D0A0000626C65206366672083
:10D3F0006E616D653A25732C206C656E3A2564006C
:10D40000617070646174615F666C6173685F757090
:10D4100064617465206E616D65206661696C656428
:10D420005B25645D0D0A0000626C65206366672001
:10D430006164765F696E74657276616C3A2564002A
:10D44000617070646174615F666C6173685F757050
:10D450006461746520696E74657276616C206661C2
:10D46000696C65645B25645D0D0A00000400FA05C3
:10D4700000ED00E070B5054601461C220E48FDF7A0
:10D48000A1FE0E4C002626702968002906D008222D
:10D49000201DFDF797FE201D7ADF02E00748001DE2
:10D4A0007BDF002807D1401E60806670044A00219F
:10D4B0000448FFF7C1FA70BDE42E00206C21002063
:10D4C00035090200000C0200F8B5214C0288002743
:10D4D0001E4DE689102A15D01E49112A21D0122A84
:10D4E0002DD0502A1CD1C288801DB24218D1428949
:10D4F000022A15D1427B037B10021843C007C00FDC
:10D500000CD112E081886980014610480822183148
:10D510000C30FDF757FE6F70002E01D100F068FB54
:10D52000F8BD0020C04368806F700868FFF722FBD9
:10D530000028F5D0A1690029F2D08847F8BD08225B
:10D54000811802480C30FDF73DFEE7E76C21002012
:10D55000E42E0020000C020010B502480068FFF71E
:10D5600009FB10BD000C02007CB5054608880C467E
:10D570000930904201D90C207CBD684671DF00283B
:10D58000FAD121880820685420881B21401C80B2D1
:10D5900020802954208800A9401C80B22080401996
:10D5A00006220131FDF70EFE20886946801D80B2FB
:10D5B00020800978002900D0012129542088401CAE
:10D5C000208000207CBD000010B50446FFF77CFFE2
:10D5D0002146054800F08EF8204601F0ABFD2046BC
:10D5E000FFF7BCFC10BD0000382600201CB5044627
:10D5F0000021684601702178817161784171A178BC
:10D600000171E178C17021798170617941705C218B
:10D6100010A0FDF718FE002805D05C210DA0FDF735
:10D6200012FE401C00E00BA0FF220146D0320DA0EC
:10D6300001F026F806212046FEF768FA01460CA004
:10D6400001F01EF80FA001F01BF86946002070DF02
:10D650001CBD00002E2E5C2E2E5C2E2E5C6D616992
:10D660006E2E63005B25735D5B25645D3A000000F0
:10D6700073657420626C65206D61632061646472FF
:10D680003A2573000D0A000030B5184B0D46041EF4
:10D690000FCB85B003936B4607C324D0002D22D057
:10D6A0000020C043A0822868A0610020A075214608
:10D6B000684663DF002814D12178684681740C49DC
:10D6C0000182A21C04A90120A0DF002809D129465B
:10D6D000204602F08DF9002803D12946204602F0A9
:10D6E000CDFF05B030BD0E20FBE70000240C02008A
:10D6F000E7FE000030B400281DD000291BD00B88A5
:10D70000102B16D00022112B17D0502B13D1CB8801
:10D71000048A891DA34202D14C89022C11D082882F
:10D72000934208D18369002B05D04A8930BC0C3163
:10D7300018478988818230BC70470021C9438182A3
:10D7400009E04B7B0C7B19022143C907C90F02D0AA
:10D7500001218175EFE78275EDE7000007B584B020
:10D7600000280DD0828A114B9A420BD0827D002A6C
:10D7700008D06A46128B142A06D9072007B000BDCC
:10D780000E20FBE70820F9E70022009201920292A6
:10D79000039282896B461A80039106A902910121A6
:10D7A0009970808A6946A6DFE8E70000FFFF000065
:10D7B0000A4610B50146024801F090FF10BD000076
:10D7C0005426002000B51C4887B04068059000230F
:10D7D00048221A4905A802F06DFA002801D0FFF787
:10D7E000C9F86A460121002002F04CFA002801D055
:10D7F000FFF7C0F8124802F071F9002801D0FFF7D6
:10D80000B9F8032069460880684602F031FA00281A
:10D8100001D0FFF7AFF80B4802F020FA002801D042
:10D82000FFF7A8F8084802F06BFA002801D0FFF7CC
:10D83000A1F807B000BD0000A40B020028240020BE
:10D84000E81F0020C9D50100BD03020002490918E4
:10D850002020085670470000202F002010B51248E5
:10D86000017842780907090F022910D8252A0ED815
:10D87000002904D001290CD05523002111E00B49C7
:10D88000801CFDF7CAFC002801D1012010BD00203A
:10D8900010BD0F23F1E74418A4789C42F7D1491C2E
:10D8A000C9B29142F7D3F0E7982D0020D80B0200BF
:10D8B000F8B53E481422017851430C18E0680C2159
:10D8C00048433A492769CC3140180589418900917C
:10D8D000241D466801F094FD01463846FDF748FCDA
:10D8E000002932D000200099A2884D436188AE19EA
:10D8F0008918CD1900222E4900280A6109D001F0AB
:10D900007FFD6188884222D0B54202D1A0880028DC
:10D910001DD0A06803281AD001F072FDA188CA1991
:10D9200001461046FDF724FC214C8808E06001F018
:10D9300067FD01462846FDF71BFC002911D0002099
:10D94000B5422FD000280ED02CE00120CBE701F00B
:10D9500057FD01463846FDF70BFC15494861032089
:10D9600021E00120ECE7ADB2B7B201F049FD01467C
:10D970003846FDF7FDFB064601F042FD014628460C
:10D98000FDF7F6FB864201D1781B09E001F038FD76
:10D99000064601F035FD01462846FDF7E9FB701A01
:10D9A00080082061022002F02FF9F8BD842F0020AA
:10D9B0008821002010B50748142201785143081827
:10D9C0000079042802D000F059F810BD012002F0BF
:10D9D0001BF910BD842F002010B50B4814220178CC
:10D9E00051430818094AC18811620079012806D0FC
:10D9F000032801D0042801D1FFF75AFF10BD0120F0
:10DA000002F002F910BD0000842F002088210020C0
:10DA100014225043054A002180180171C18002225E
:10DA20000161C2604161018170470000842F0020C4
:10DA3000F8B5104C069E65780A2D19D027787D1907
:10DA40000A2D00D30A3D14277D432D1928716A61E0
:10DA500003C92961E860EB802E816078401C60700A
:10DA600005480078002801D1FFF7B6FF0020F8BD77
:10DA70000420F8BD842F00208821002010B50D4C13
:10DA800014212078484301190020091DFEF7A8FF42
:10DA90002078FFF7BDFF6078401E60702078401C42
:10DAA000C0B220700A2801D100202070002002F0AE
:10DAB000ABF810BD842F0020F8B52348C1680029B9
:10DAC0003ED00E6821494C680769C078E11B0D0201
:10DAD0002D0AED1C002814D101201D4A00045060BD
:10DAE0001B4A403A50601B49400008601A490860D0
:10DAF0001A49012008602F20FDF70EFB1249012072
:10DB0000C870B54200D23546E81900020F4B000A32
:10DB1000403318600D4A5168001B091B0902090AAD
:10DB20000002000AC91C814209D9506818602F20E0
:10DB3000FDF7F2FA01200749400480390860F8BD7A
:10DB400001F018FFF8BD0000D821002000150140A9
:10DB50004013014080E200E000E100E000100140DD
:10DB6000F8B50646108814468446801D0D46984236
:10DB700001D90C20F8BD32880720062AFAD31927CC
:10DB8000FF01184BBA4201D99A42F3D17188062994
:10DB9000F0D3B94201D99942ECD19A4203D09942CB
:10DBA00001D08A42E6D805216046295420881221F6
:10DBB000401C80B2208029542088401C80B22080E4
:10DBC0004119308802F0B0FE2188401880B22080D0
:10DBD0004119708802F0A8FE21884018208000209A
:10DBE000F8BD0000FFFF000010B5FEF7C3FE10BD3A
:10DBF000F8B5164800F0A2FB144D00260C3D144C5D
:10DC0000002807D0616900291CD001206A461070E5
:10DC1000684616E02878002805D06169002911D0EF
:10DC2000684606700DE0687800280DD0A1680948A4
:10DC300000220068FEF760FF002803D0A1690029D8
:10DC400000D088472E70F8BD6168F0E77821002089
:10DC5000E42E0020000C020010B5134C20790007C0
:10DC60001FD46069401C6061E068002801D0042076
:10DC700004E000F095FB002803D0022002F094FBA2
:10DC800010BD2069002809D06068C10701D00320B9
:10DC9000F4E70121084360600020EFE7FFF78AFE08
:10DCA00010BD02F075FB10BD8821002010B508489A
:10DCB00041680A0708D48A0702D50122114341604E
:10DCC000022002F071FB10BD02F062FB10BD0000EB
:10DCD00088210020F8B51646424CD2B2A272A36346
:10DCE0000125E16365720027E7812778002F08D0BE
:10DCF000002808D0032809D0012F0FD0E581022089
:10DD0000F8BD0520F8BD00F03DF968E0012FF5D021
:10DD1000A0890121C9030843E081F4E7272902D93A
:10DD2000E5810120F8BD0027A781012802D0022843
:10DD300009D054E027212C48FDF75DFA012001F0BD
:10DD400087FD04202CE0252A02D9E5810320F8BDB7
:10DD50001F073F0F24485B1C0770244F427021D0DF
:10DD6000012B05D0022B09D0032B09D0E58130E02F
:10DD700032461F49801CFDF725FA06E00F2200E01D
:10DD800055223146801CFDF72FFA002001F060FD7E
:10DD9000A1691848FF3141310161476145600220A6
:10DDA00020701CE00846002E06D0012E04D0022E62
:10DDB0000CD0032E13D10EE0002001F049FD0E49D6
:10DDC000032008600D490D603D60E9E700F0C8F8E8
:10DDD00003E00420F8BD00F0A1F80028F9D00020ED
:10DDE000F8BD00000C210020982D002000100040FC
:10DDF000D80B020000F50140401500400012004021
:10DE000010B5810402068307840B890E920E9B0FC6
:10DE1000032B00D11B1F2046FFF75CFF10BD000045
:10DE200010B502F0E5FA002803D101F0B3FC002898
:10DE300001D0042010BD064800214172012101706B
:10DE400004480169102211430161002010BD000047
:10DE50000C21002000ED00E090B00E46074601F0D6
:10DE600075FDFFF7DDFF002211460C2002F040F99E
:10DE70000025284C0EE0384601F01CFC002809D192
:10DE80006946384601F061FC002803DD81B268462E
:10DE900002F0DAF8384601F00DFC0028EBD03046ED
:10DEA00001F008FC002809D16946304601F04DFC1C
:10DEB000002803DD81B2684602F01EF820780228AF
:10DEC00002D0032809D012E0134825700088FFF71C
:10DED00097FF002211460E2007E0032025708003E3
:10DEE000FFF78EFF002211460F2002F001F938469D
:10DEF00001F0E0FB002809D16946384601F025FC15
:10DF0000002803DD81B2684602F09EF800F04EF86A
:10DF1000C5E7000082200020F82000200C490A7884
:10DF2000012A05D8002805D0012807D0022809D0E9
:10DF30000020704707488861082006E0064888618D
:10DF4000092002E0054888610A20487001207047D6
:10DF50000C210020008000400090004000A0004004
:10DF6000074942B20B78012B04D828322D2A01D25E
:10DF7000820701D0002070474861012070470000EF
:10DF80000C21002010B50649002008600549012435
:10DF90008C600861486101F087FC0348047010BD83
:10DFA0004015004000F501400C210020F8B51E4846
:10DFB00001691022114301611C4F01251C4C0026F0
:10DFC000F868002817D0FE601A4802210160207806
:10DFD000042810D11848456018480068012806D167
:10DFE000FFF73CFC002802D0A089401CA08127211B
:10DFF0001348FDF700F9A069FF300130016C0029DA
:10E0000001D00664DCE7406C0028D9D0A069FF305D
:10E01000013046646078C006C00E85400548056042
:10E020002069401C2061F8BD00ED00E000110040B7
:10E030000C21002080E200E00010004000140040AD
:10E04000982D002010B50E4900234A788C78A24202
:10E0500012D0521CD2B24A70022A00D14B704A78B8
:10E06000074B920018339A58026008691018000292
:10E07000000A0861012010BD0360002010BD0000EF
:10E08000D8210020826883881A4003689A5C0A704D
:10E090008168491C81607047C26883881A400368A0
:10E0A0009954C168491CC1607047000010B5002830
:10E0B00003D0112802D0FEF7AFFC10BD02480822A1
:10E0C00041681143416010BD8821002010B51C4CEF
:10E0D000217820464068012906D0022929D0032949
:10E0E00012D1000717D513E0000711D415481422E8
:10E0F000017851430818C188A28B891A0904090CB8
:10E10000C18002D002F008F910BDFFF7B7FC10BDC6
:10E1100000F004FC10BD6069401C606100F040F933
:10E12000002803D0207801F06FFD10BDFFF742FCFE
:10E1300010BD6078044980000858804710BD000079
:10E1400088210020842F0020880C020010B528DFD1
:10E15000FFF7ACFF10BD10B529DFFFF7A7FF10BD1B
:10E1600010B50446C0B2FEF77FFD204610BD00008A
:10E17000002804D00349496D016000207047032046
:10E1800070470000803000203EB520480546FDF76E
:10E190003DF8082800DD0820044669461120087271
:10E1A0005C211BA0FDF74FF8002805D05C2118A0CA
:10E1B000FDF749F8401C00E015A00146872218A091
:10E1C00000F05EFA294619A000F05AFA1BA000F0F0
:10E1D00057FAA2B2294602A87CDF002000900C2248
:10E1E000694601900A8028224A808880FF20913069
:10E1F000C88068467ADF002801D0FEF7BBFB042008
:10E2000077DF002801D0FEF7B5FB3EBDBC20002023
:10E210002E2E5C2E2E5C2E2E5C6D61696E2E6300A0
:10E220005B25735D5B25645D3A00000073657420B7
:10E23000626C65206E616D653A2573000D0A000001
:10E2400001480078704700000821002070B51B4C81
:10E25000207900072ED41A481422017851430D1852
:10E260002E6901F0CDF80146E8882A89761E8018CB
:10E270008019FCF77DFF21690025002909D061691B
:10E28000814206D1E560606801210843606000209A
:10E290000AE000F085F8002802D00220E56003E0E3
:10E2A0002069002803D0032002F07EF870BDFFF73C
:10E2B00081FB70BD02F06CF870BD00008821002069
:10E2C000842F0020F8B51C4C2078002833D020691A
:10E2D000002807D00026E068002805D00025002E81
:10E2E00004D011E00126F6E70125F8E7684652DF81
:10E2F000052804D0002804D0FEF73CFB04E00126EA
:10E3000002E0216900988847002D10D16088694695
:10E310000880A06861DF052804D0002804D0FEF73B
:10E3200029FB04E0012502E0E168A0688847002E8F
:10E33000DCD0002DD3D0F8BDBC2100204188054899
:10E340000288914204D34088814201D8012070475D
:10E3500000207047702100201048018CC9B20129AB
:10E3600017D1818C090714D1018D09060A0F03D139
:10E37000828D1206120F0ED0090F012903D1828D52
:10E380001206120F07D0032903D1808D0006000F5B
:10E3900001D000207047012070470000C00F00F03E
:10E3A00070B50E481422017851430C18256901F00C
:10E3B00027F80146E08822896D1E80184019FCF775
:10E3C000D7FE07494A69824206D3824202D10869D0
:10E3D000002801D0002070BD012070BD842F0020D6
:10E3E00088210020800701D000207047012070475D
:10E3F00030B51588EC1C9C4201D90C2030BD02249C
:10E400004C5513881C255B1C9BB21380CD5413887C
:10E410005B1C9BB21380012807D0022807D0032879
:10E4200007D0042807D0072030BD002004E00120D9
:10E4300002E0CC5401E00320C8541088401C108036
:10E44000002030BD01490320086070477407005068
:10E45000002803D10120024940078860704700006E
:10E460000005005010B5C821024802F05BF80249CF
:10E47000087010BD99E4010080200020002808D118
:10E4800004480121426849070B46934383600A40D0
:10E49000C26070470005005010B50020FFF7EEFF86
:10E4A00010BD0000F8B52C49C8680A690C780F79CE
:10E4B00089688646944600913EE00099E20055182E
:10E4C0002A7836E0182353436968521CC918AB7880
:10E4D000D2B2934200D100220B78022B02D0032B40
:10E4E00027D123E04E680346014603E0B14204D041
:10E4F0000B46C96900291CD0F8E7002919D08B42C6
:10E5000008D1C069002805D1144F0126BE6000263D
:10E51000B44601270E68C969D961002909D00B6882
:10E520009B190B6005E00174C06900E00021002820
:10E53000F9D169789142C5D12146641EE4B200291F
:10E54000BBD1054962460A61C8600F71704501D0B0
:10E550000120F8BD0020F8BDD821002000100140A6
:10E56000F8B5044631480026C168009107784EE0AE
:10E570002E48F90080680D1843E0002C02D0204698
:10E58000E4691FE02878182141436A68401CC0B242
:10E5900051182870AA78904200D12E700A784868E5
:10E5A000012A30D1027C002A2DD18A684260CA68D3
:10E5B00082600A69C260496981611C490979002940
:10E5C00000D04660194943680A699C46991A0902B5
:10E5D000174B090A994202D28268891807E06146FE
:10E5E000511A09028268090A8A4202D9511A016045
:10E5F00000E006604660012186600174C66101F09A
:10E6000071FF002CB9D1287869788842BAD1384690
:10E610007F1EFFB20028ABD10448C1680098814238
:10E6200001D00120F8BD0020F8BD0000D821002055
:10E63000FFFF7F0030B50E4C87B02078002802D055
:10E64000002007B030BD0B4A04AB07CA07C3084817
:10E650000125401C009008480290802003900195FD
:10E660000323064A694604A8FEF7AEFA2570E8E7D8
:10E67000FC210020C00C0200D83000203D07020021
:10E680000FB410B503A90298FDF700FB10BC08BC3D
:10E6900004B0184730B5002391B07B4A05211846D5
:10E6A000FEF7E2F9002801D0FEF764F9774801F09F
:10E6B00042F8774801F03FF8764801F03CF8FFF760
:10E6C000B9FFFFF7BFFE0020FFF7C2FE7249734893
:10E6D00001F008FC02F03AFA02F02EFA01F078FBA1
:10E6E000FFF770F8FEF710FB00223C216C48FEF7A4
:10E6F00027FB5C216BA0FCF7A6FD002805D05C2160
:10E7000068A0FCF7A0FD401C00E066A08322014643
:10E71000920068A0FFF7B4FFFFF792FD014668A3DF
:10E720006AA26DA0FFF7ACFF71A0FFF7A9FF5C48DC
:10E73000203001790446303CFF290CD04179FF2973
:10E7400009D057497D22898CD200E180914202D9BB
:10E75000FF214131E180007B0025FF2806D1504890
:10E76000E56364A12C302564FCF764FD634A012154
:10E770006348FEF761F9002801D0FEF7FBF8604816
:10E78000002221210068FEF7B7F9002801D0FEF72A
:10E79000F1F8434808213430FEF728FFFFF7F4FC76
:10E7A00058480090394869461C38FEF76DFF00282C
:10E7B00001D0FEF7DFF8FEF713F81C216846FCF7DE
:10E7C0001AFD0520C00301900F200004029000955F
:10E7D000032168460173C58105744B4805904B4879
:10E7E00006906846FEF746FE002801D0FEF7C2F804
:10E7F0000320FEF711FC002801D0FEF7BBF8FFF75D
:10E8000031FE4349434801F08DFE7D210901424814
:10E8100001F088FE60701F4800F04CFF002809D10D
:10E8200069461C4800F091FF002803DD81B268466C
:10E8300001F062FBA07801281ED0144800F03AFFD6
:10E84000002809D16946114800F07FFF002803DD48
:10E85000C1B26846FDF774F80D4800F02BFF0028A0
:10E86000D9D169460A4800F070FF0028D3DD81B293
:10E87000684601F0E9FBCEE706490548FFF7ECFAE8
:10E88000002011B030BD000070240020542600206C
:10E8900080280020AC2A002021FD0100B1D7010012
:10E8A000902000202E2E5C2E2E5C2E2E5C6D616939
:10E8B0006E2E63005B25735D5B25645D3A0000008E
:10E8C00030303A33303A3338000000004A616E206D
:10E8D00031312032303233005645523A5B253032E6
:10E8E000585D2C4275696C643A25732025730000CD
:10E8F0000D0A00003133646F67000000E903020075
:10E90000A40B0200A9F001009DF20100E9DB010067
:10E9100088130000D5F20100E5F8010010B50448A5
:10E920000822416891434160007801F06DF910BD03
:10E930008821002030B5084A084B08E00578140A01
:10E9400055402A06D20D9A5A401C6240491E0029A1
:10E95000F4DCD04380B230BDFFFF00000422002071
:10E9600070B5144682880E4605462088111D411850
:10E97000921C994201D8FE2A01D90C2070BD521C6C
:10E9800032542088FF21401C80B2208031542088DE
:10E99000401C80B220808119288801F0C5FF2188A1
:10E9A000401880B22080AA88002A09D0A9680029CE
:10E9B00008D08019FCF706FC2088A9884018208020
:10E9C000002070BD072070BDF8B50F4601781446D1
:10E9D0000546012902D16878002806D02088821CCB
:10E9E0009A422DD8012902D006E00720F8BD6978A7
:10E9F0004118891C994223D8181A801E86B268468D
:10EA000006802188B81C081869467DDF0028EDD1F2
:10EA10002878022805D169460988B14201D8092120
:10EA20000AE00821012805D16878B04202D86A4678
:10EA3000108001E06846068068460088FE2801D9FB
:10EA40000C20F8BD2288401CB8542088401C80B29D
:10EA50002080395420886946401C2080098840184D
:10EA600020800020F8BD000031B5054C04E0401EB8
:10EA700000902046FCF740FB00980028F7D138BDF5
:10EA8000E70300008207D30EFF229A408907090E90
:10EA900010B5994000280BDA03071B0F083B9C08B0
:10EAA0000C4BA400E318DC6994430C43DC6107E0E1
:10EAB0008408094BA400E418236893430B432360A4
:10EAC000C106C90E01208840044908600449086055
:10EAD00010BD000000ED00E000E400E080E200E096
:10EAE00000E100E0400F012800D000207047000046
:10EAF000FFB506460F46007918214843184981B0F2
:10EB000044181D46002B18D0002F16D03846FFF7AA
:10EB1000E9FF002813D02846FFF7E4FF00280ED0B5
:10EB2000607D00280DD0012818D0022809D00328C4
:10EB300007D00325284605B0F0BD0E20FBE71020C6
:10EB4000F9E7E7602561039820600A986060002576
:10EB500001222146306801F09DFAEBE70825E9E73C
:10EB600068300020F7B507460C4600791821484365
:10EB70004C4986B041180491097D3E68002902D0B5
:10EB8000082009B0F0BD002C01D147494418207C71
:10EB9000032801D90720F4E7089800280DD0206841
:10EBA0000025FF280BD0E17C002300911A46019537
:10EBB000194600F027FA206803E00E20E1E7002064
:10EBC000C04302906068FF2808D0002300951A46D1
:10EBD0001946019500F016FA606801E00020C04374
:10EBE0000095019503900022A37C1146E06800F097
:10EBF00009FA0023009501951A461946A06800F00D
:10EC000001FAE068A3688446052000023018039AE0
:10EC10000299009083600261C1606246426145636F
:10EC2000856345648564607C217C002800D00120D8
:10EC3000012904D0022904D0032906D103E00221CE
:10EC400002E0042100E0062108430099486500998C
:10EC5000207DC8650B21C901607D71180864FF2003
:10EC600005303550FF20293035503979182041437F
:10EC70000C4809184D753979182359430818089A12
:10EC8000826059010948711848600520A17D3856F5
:10EC9000FFF7F8FE04980121017500990220086031
:10ECA00000206EE7683000209C0C02000204000087
:10ECB000F3B52A4C0746E07E81B0002801D0082039
:10ECC000FEBD002F00D1264F012638783146814005
:10ECD00024488160386800F0B0F90021786800F0BD
:10ECE000A3F9214DB8696862787D397D0843E866EB
:10ECF00003CFE8606961387B083F01280FD100210C
:10ED0000B86800F091F9387B314681401548816040
:10ED1000F86800F092F9F968B868A960286102986B
:10ED200060603969216000280ED0FF230F481D3331
:10ED3000397F0022C250FF234533C2500D4A0C4890
:10ED400050600220FFF79EFE042028600020E0753E
:10ED50002076A075E676A076FEBD0000682F002024
:10ED6000540C020000050050002500400020004027
:10ED70008000020000230040F8B5104B81245E683B
:10ED80000022A4000E4D002E00D0AC60DF7D002FCD
:10ED90000BD01A7E002A04D0002E00D06C60112007
:10EDA000F8BD18610122197604E0D9750024D860F5
:10EDB0005C761C7600F012F8F8BD0000682F002089
:10EDC0000023004010B5044CA07E002803D100F0C1
:10EDD00077FE0120A07610BD682F0020F8B5234DE6
:10EDE000A87E104301D100F06BFE6868204C00281B
:10EDF00005D081201F49800048600020F8BDFF2019
:10EE0000453000212150FF212531204600F03FF9F7
:10EE10000546FF210931204600F039F90746FF2158
:10EE20004531204600F033F906463946314329433F
:10EE3000E9D02846304306D100F0BEFD0B48C17D25
:10EE4000407E8142DFD800210848002DC17501D0E5
:10EE50000320F8BD002E01D00F20F8BD817E0120D7
:10EE6000002901D02060C8E76060C6E7682F002055
:10EE7000002000400023004010B5034600F048F891
:10EE8000002801D0112010BD034A00209175936025
:10EE9000908200F003F810BD682F0020F8B500261E
:10EEA000194FFF251D357E510120B86001F0D0FBC0
:10EEB000164C6168002910D022E0FF27013729464F
:10EEC000114800F0E4F8002802D1A08AB842F6D137
:10EED000A08AB84201D001F0BBFBA08AA17D884284
:10EEE000EBD3A18AC81FF9380CD0074F2946384602
:10EEF00000F0CDF80028F9D00120F8600020A075BE
:10EF00003046F8BD0F26F9E700200040682F0020AA
:10EF10000248807D002800D001207047682F002023
:10EF200038B504460020694608706846FDF7B8FE0B
:10EF30000A48816808290AD221704A1C8260084860
:10EF4000826801238B401A438260002400E004247D
:10EF500068460078FDF7C2FE204638BDB02100208B
:10EF600000050140034A8000014980180160704794
:10EF70003546526E000601400449012048600146B2
:10EF800003480160034902200870704700030140F4
:10EF900000000140B021002070B504460D484160DA
:10EFA0000178002901D0082070BD01210170002CDA
:10EFB00000D1094C094D2078E86060687D21C003CC
:10EFC000C900FCF7D5F86860217A1020FFF75AFDD8
:10EFD000002070BDB0210020B40C020000050140EB
:10EFE00030B552000A439900039C0A432102049D54
:10EFF0000A4329040A43024980004018026030BDD8
:10F000000007005030B552000A439900039C0A43A0
:10F010002102049D0A4329040A4302498000401842
:10F02000026030BD000700501CB500220B46009264
:10F0300011460192FFF7D4FF1CBD1CB500210091C1
:10F040000B46012201911146FFF7CAFF1CBD0000CB
:10F05000820006481018026803231B049A430260CA
:10F06000026809040A43026070470000000700506C
:10F07000034940180068012800D0002070470000B4
:10F08000006000404058002800D0012070474058E0
:10F09000002800D001207047032212028018406827
:10F0A000084000D00120704770B50D4614465C2121
:10F0B00011A0FCF7C8F8002805D05C210EA0FCF7D1
:10F0C000C2F8401C00E00CA001469B220EA0FFF7F6
:10F0D000D7FA21462846FCF719FD014622460DA025
:10F0E000FFF7CEFA11A0FFF7CBFA224629460320FC
:10F0F00000F0FEFF70BD00002E2E5C2E2E5C2E2E2A
:10F100005C6D61696E2E63005B25735D5B25645DDC
:10F110003A000000626C655F72785F646174613A06
:10F1200025732C6C656E3A25640000000D0A000002
:10F1300070470000FEB5404E0446051D0188B088AA
:10F14000132974D011DC01291DD010291CD01129DC
:10F1500019D15C2139A0FCF776F800284DD05C214C
:10F1600036A0FCF770F8401C48E01B290BD01D2985
:10F1700009D0522907D100231A461946A9DF0028D1
:10F1800001D0FDF7F7FBFEBD5C212CA0FCF75BF87E
:10F19000002805D05C2129A0FCF755F8401C00E0B0
:10F1A00026A00146E32229A0FFF76AFA29882AA0AF
:10F1B000FFF766FA2EA0FFF763FA1F4801F030FA56
:10F1C000A088B080002100910191684602910170F1
:10F1D0000122427081700621C170A17B0171617BA7
:10F1E0004171217B8171E17AC171A17A0172617AE9
:10F1F00041720A220146042015E010A00146F622C1
:10F2000012A0FFF73DFA2A7929881AA0FFF738FAE9
:10F2100017A0FFF735FAFFF725F90020C043B080AB
:10F2200000221146052000F063FFFEBDFFE700232A
:10F230001A4685217FDFA2E7802000202E2E5C2E3B
:10F240002E5C2E2E5C6D61696E2E63005B25735DF6
:10F250005B25645D3A000000626C6520636F6E6E32
:10F2600065637465642C68616E646C653A2564003E
:10F270000D0A0000626C6520646973636F6E6E65D1
:10F28000637465642C68616E646C653A25642C72E5
:10F290006561736F6E3A30782578000010B500789C
:10F2A000002807D104483B21808876DF002801D060
:10F2B000FDF760FB10BD0000802000200021425CB3
:10F2C000002A01D001207047491C0629F7D30020ED
:10F2D0007047000010B5124C5C21E068401DE060F2
:10F2E00010A0FBF7B0FF002805D05C210DA0FBF7B4
:10F2F000AAFF401C00E00BA0014665220DA0FFF70D
:10F30000BFF90FA0E168FFF7BBF912A0FFF7B8F94A
:10F310001149E068884201D10020E06010BD000082
:10F32000802000202E2E5C2E2E5C2E2E5C6D6169BE
:10F330006E2E63005B25735D5B25645D3A00000003
:10F34000626C652072756E207365636F6E64733ACC
:10F35000256473000D0A0000803A09000749097905
:10F36000490701D408207047002804D0044949788F
:10F370000160002070470E207047000088210020A7
:10F38000842F002070B5134B1B795B0701D4082034
:10F3900070BD002817D0002A15D00368022B10D2A8
:10F3A0000C240D4D5C432E59002E0AD0466860197E
:10F3B000048945894068614365437118281888426B
:10F3C00003D8072070BD0E2070BD1360002051606F
:10F3D00070BD0000882100205030002010B5074883
:10F3E0004469601C06D000F00BF801462046FBF78C
:10F3F000BFFE10BD01200007406910BD00100010C5
:10F4000001200007006980B27047000070B5002439
:10F4100014482546047044702846FEF7F9FA6D1C1E
:10F420000A2DF9D3104D6C80FFF7D8FFC61EFFF7E9
:10F43000E7FF46430B4A0020AE60CC326C610C21E2
:10F440004143545089180C81401C4C810228F6D34A
:10F450000548243004602C70AC610420EC616860C5
:10F46000002070BD842F002088210020FFB528488F
:10F4700081B000791F4616460C46400702D408208A
:10F4800005B0F0BD002C1DD0019800281AD02068CE
:10F49000022815D20C211F4D4843295800290FD0AE
:10F4A00041194A8908894968424351186268914262
:10F4B00006D9002E04D0B04202D3F119814203D9FB
:10F4C0000720DDE70E20DBE70198FEF78BFF002821
:10F4D0001BD03846FEF786FF002816D06068FEF77E
:10F4E00081FF002811D060683246C1190198FBF7EE
:10F4F00069FE009620680C2148432D580022022105
:10F500002046019BA8470020BAE71020B8E700007A
:10F510008821002050300020F8B52C4D0446287971
:10F520000E46400701D40820F8BD002C20D0002E44
:10F530001ED0206800281BD0FFF762FF0146A0887C
:10F54000814213D3102811D3E08800280ED0FFF792
:10F5500045FF471EFFF754FF4743E288A188A8688C
:10F560004A431218974201D3890703D00720F8BDF8
:10F570000E20F8BD6988022926D031600C22144B78
:10F5800051437060CA18506020685850A08810819C
:10F59000E0885081FFF734FF0646FFF731FFA1886E
:10F5A000E288401E514340183146FBF7F7FD044600
:10F5B000FFF726FF0146A86861430818A86068881D
:10F5C000401C68800020F8BD0420F8BD8821002080
:10F5D0005030002010B5114902460878002811D09B
:10F5E00004280FD0022A16D0032A0BD10A79120759
:10F5F00011D48A69521C8A61032A08D0022802D0D9
:10F6000000F002FB10BD487800F0CEFE10BD0D20CA
:10F61000FDF702FA10BDFEF759FD10BD882100204C
:10F62000F8B5044621481E46007915460F464007A6
:10F6300001D40820F8BD002F1CD0002C1AD021685E
:10F64000022915D20C20414319484258002A0FD0F4
:10F6500008184289018940684A431018626890423C
:10F6600006D9002D04D0A94202D3A819884203D993
:10F670000720F8BD0E20F8BD3846FEF7B3FE00287F
:10F6800011D03046FEF7AEFE00280CD06068FEF7C1
:10F69000A9FE002807D02B463A46214604200096B2
:10F6A000FEF7C6F9F8BD1020F8BD00008821002043
:10F6B00050300020FF30FF300230806A002801D037
:10F6C0000020704701207047FF30FF300230806A11
:10F6D000082801D00020704701207047F8B50F4678
:10F6E0000546FFF7F1FF002824D1402A00DD402223
:10F6F000EC1DFF34FA34606A1646401CC117490FEE
:10F700000918C908C900401A6062A16A491CA162AF
:10F71000442148434019FBF76EFD606A4421484389
:10F72000401932463946001DFBF74CFD606A442102
:10F7300048432E50F8BDFF300021FF30C94302304E
:10F740000162416200218162704770B50B46054637
:10F75000FFF7B0FF002801D0002070BDEC1DFF3482
:10F76000FA34206A401CC117490F0918C908C9009A
:10F77000401A2062A16A491EA162442148434119EE
:10F780002A581846091DFBF71DFD206A44214843ED
:10F79000285870BD10B52A48C06A00070CD4284804
:10F7A0004030C26A27494A62026B8A62426BCA626F
:10F7B000826B0A63C06B4863234CFC22606901467C
:10F7C000914308D140B2042805DC2821C84202DB5D
:10F7D000207A032801D9042010BD00F065F81B48E9
:10F7E0006169C160217A0161416A090A09024162C5
:10F7F000426AA16A0B0E1A4342620902C1610121E9
:10F8000001630021C1626179E27909021143416318
:10F810002179E278090412021143A278114341616F
:10F82000A18C228C490612061143A28B12041143AB
:10F83000A2791202114325318161002010BD000020
:10F8400080000010001700400C210020001500402F
:10F8500070B50F4900230B600E4A0D49D46A403938
:10F860008C63146BCC63D46B6400A41C8C600A4C56
:10F870004C600A4C23600A4E03253560002804D0F2
:10F88000E36008490120486070BD5069C86070BDE0
:10F89000401500400C210020982D00200011004050
:10F8A0000012004000100040094903208860094907
:10F8B0000020086008490861084A012313610B69A8
:10F8C000002BFCD0086150601060054988817047AA
:10F8D00000F50140001200400011004000100040FF
:10F8E0000C21002010B55C210CA0FBF7ACFC00281B
:10F8F00005D05C2109A0FBF7A6FC401C00E007A096
:10F9000001466E2209A0FEF7BBFE0BA0FEF7B8FE73
:10F910000DA0FEF7B5FE00F059FC10BD2E2E5C2E9A
:10F920002E5C2E2E5C6D61696E2E63005B25735D0F
:10F930005B25645D3A0000007265706F727420761A
:10F940006572206E6F7700000D0A000010B5FDF79C
:10F9500003FE002801D0FDF70DF874DF00F0C4F9B4
:10F96000002801D0FDF706F87D20C000FFF77CF8E5
:10F9700010BD000070B501240B49600408600B49FC
:10F9800040108860094940398860094D6C602F201B
:10F99000FBF7C2FBAC60074D00242F202C61FBF766
:10F9A000BBFBEC7070BD000080E100E04013014043
:10F9B00000100140D821002030B50A48FF21C57D44
:10F9C0000022094C0931094B002D625007D099697A
:10F9D000437EC268D154417E491C417630BD98694E
:10F9E00030BD0000682F00200020004000250040AE
:10F9F00070B50546294894B00FC800240AAE029499
:10FA00000FC6601C0007000F694610300872601CAA
:10FA10000007000F10304872887AF9263040801CA9
:10FA200088721C2103A8FBF7E6FB6946087B1221BC
:10FA300008436946087302A8049408900694079442
:10FA4000294609940AA863DF002825D128786A4648
:10FA5000907113489080112000941070507090782D
:10FA6000F7213040801C0840EF2108400126304338
:10FA7000907014210EA8FBF7BEFB01A80E906846FB
:10FA80000F9010AA16801420548090802B4668880E
:10FA90000C330EAA03A9A2DF14B070BD040C02003F
:10FAA000F63600001FB501236A4613701072034832
:10FAB000019106C8684690471FBD0000682F0020CE
:10FAC000FF220548253200218150FF220932815052
:10FAD00001210160704700000020004008B5024984
:10FAE0000020009108BD00008020002010B50121F9
:10FAF000202805DA1A4A8140114201D1194810BD67
:10FB00008107C90E002808DA0207120F083A920886
:10FB1000154B9200D218D26904E08208134B920070
:10FB2000D2181268CA401106890F042911D200297F
:10FB30000FD002290DD00E494C68C306DB0E0122FE
:10FB40009A40002C08D0400980000B5813430B50FA
:10FB500004E00448401C10BD06480260002010BDAF
:10FB6000FC06FFBC0120000000ED00E000E400E026
:10FB7000D021002000E100E0FFB50746806A81B097
:10FB8000144600283DD0002538462030009033E050
:10FB90000C20B96A68430E18B088801CFE2802D970
:10FBA0000C2005B0F0BD22880299401C88542088A2
:10FBB0001622401C80B2208002990A542088401CE2
:10FBC00080B2208002994118308800F0ADFE218873
:10FBD000401880B22080B288002A0AD0B16800297B
:10FBE0000FD0029BC018FBF7EDFA2088B1884018AF
:10FBF00020806D1C0098EDB2007BA842C8D8002080
:10FC0000CFE70720CDE7000010B50F4900280870A6
:10FC100009D0012811D0022812D0032802D1486946
:10FC2000FEF794FA10BD00208861C861074840784B
:10FC30000028F7D0FDF7D0FE10BD00F06DFB10BD21
:10FC400000F0CEFA10BD000088210020842F002093
:10FC5000017842780270417070470000002803D09C
:10FC60000249C860002070470E207047BC21002068
:10FC70001CB5034901910091694660DF1CBD00007D
:10FC80008020002070B50E4605461446142110460B
:10FC9000FBF7B1FA01200021208021612173267237
:10FCA0006572002D00D0A072002070BD10B5FCF769
:10FCB00053FE10BD70B5002901D08C0701D007207C
:10FCC00070BD074C0125A16062800649636010DFAA
:10FCD0000028F5D125701620FFF708FF70BD000041
:10FCE000BC210020ADFC010011DF002801D0012162
:10FCF00000E00021014A117070470000BC21002083
:10FD0000002803D002490861002070470E20704788
:10FD1000BC210020417800780002084370470000B1
:10FD20000A4610B501460248FFF7D8FC10BD000096
:10FD300080280020F8B506460C468A1815E02046B3
:10FD4000FFF7E8FF0746A41C2046FFF7E3FF054640
:10FD5000A01C441994420BD8B74206D101462A464A
:10FD60001846FBF72FFA2846F8BD201D9042E6D929
:10FD70000020F8BD07B56846007801281DD110485D
:10FD800042780121002A04D0002242700D4B20222B
:10FD9000DA60019A002A10D00B4A1378002B02D1A6
:10FDA0005278002A0AD0017007490848019AFFF7E3
:10FDB00095FC40210448FBF71EFA0EBD8170F8E760
:10FDC000CC20002000050050182D0020AC2A002077
:10FDD00070B50225164888B0032404600126154931
:10FDE0002020C8601822144901A8FBF7EBF9042071
:10FDF000049001A970C168468475C47504750E48E5
:10FE00000E4A01A90838FEF7ADFE002801D0FCF724
:10FE1000B1FD40200A4B0246191A009006480838E6
:10FE2000FEF766FE002801D0FCF7A4FD08B070BD07
:10FE30001407005000050050B40B020075FD0100CE
:10FE4000182D0020FEB50D46FF2104462931FFF78D
:10FE500019F90521090200276618002816D0FF208D
:10FE600029302750687D012810D1E968286871641D
:10FE7000C0B2B064296968687163C0B2B063012020
:10FE8000A06202222946204600F004F9FF21053134
:10FE90002046FFF7F7F8002814D0FF200530275040
:10FEA000012069460870F06BC0B20190F06CC0B2DE
:10FEB0000290A868002801D1FCF75CFD6C4607CCD5
:10FEC000AB689847FEBD000004484178002904D083
:10FED0000021417002492020C8607047CC200020DA
:10FEE00000050050002804D0002902D0014A91608A
:10FEF00050607047FC200020F8B5044640213B4884
:10FF0000FBF779F9A578E778681EC6B23146A01CE0
:10FF1000FEF710FD0346A1198A7868460270C97879
:10FF20004170FFF795FE68460088834215D1E0785E
:10FF3000012812D02E4E032F10D0072836D00928C2
:10FF40003FD02C490C2843D00E2843D00F2844D052
:10FF50000B2844D028A0FEF793FBF8BD5C212CA011
:10FF6000FBF771F9002805D05C2129A0FBF76BF99C
:10FF7000411C00E026A17A2229A0FEF781FB201D6A
:10FF8000E91EFBF7C3FD0146EA1E28A0FEF778FB39
:10FF90002CA0FEF775FB211DEA1E1448FBF712F991
:10FFA000ED1E7268E9B211489047F8BD211DEA1EA6
:10FFB0000E48FBF707F9ED1EA9B20C48FDF722F930
:10FFC000F8BD30780028FBD000221146092009E056
:10FFD000012000E002200870F8BD0320FBE70022AA
:10FFE00011460B2000F084F8F8BD0000582D0020C9
:10FFF000FC200020822000205350492050726F6363
:020000040002F8
:10000000657373204E6F6E2044617461200D0A0089
:100010002E2E5C2E2E5C2E2E5C70726F632E630073
:100020005B25735D5B25645D3A000000636D645F72
:100030007472616E736665723A25732C6C656E3AE4
:10004000256400000D0A000070B506460E4C002025
:100050000D46A0707D20C000606040210B48FBF77A
:10006000CAF82A4631460948FBF7ACF8012060700F
:10007000074920208860A078002803D1FCF794FA73
:100080000028F8D070BD0000CC200020D82C002023
:100090000005005010B54A7500F001F810BD3EB5DE
:1000A0004A7D0C460121012A16D0022A16D0032AC5
:1000B00011D16A461170052109024018C16BC9B2FD
:1000C0000191C06CC0B20290A06800280BD06D46B0
:1000D00007CDA36898473EBD41623EBD00206946FA
:1000E00008700190EFE70020FCF744FCEFE7000008
:1000F00070B590B00E460446154640216846FBF7A1
:100100007AF8FFF7E1FE40216846FBF774F8F1202A
:10011000694608704870E81C8870CC700C46002D49
:1001200006D03A2D04DC081D2A463146FBF74AF872
:100130002D1DA91EA01CFEF7FDFB010A6155291902
:100140004870AD1CACB25C2111A0FBF77CF8002814
:1001500005D05C210EA0FBF776F8401C00E00CA057
:1001600001463F220EA0FEF78BFA21466846FBF7B8
:10017000CDFC014622460DA0FEF782FA11A0FEF743
:100180007FFA114AE1B292686846904710B070BD9C
:100190002E2E5C2E2E5C2E2E5C70726F632E6300F2
:1001A0005B25735D5B25645D3A0000007370695FD9
:1001B00074785F646174613A25732C6C656E3A25BE
:1001C000640000000D0A0000FC20002008B5FEF7C6
:1001D00037F86946087001221046FFF789FF08BD0D
:1001E000F8B5164C1422606840084000606014485E
:1001F000017851430E183769FFF702F90146384676
:10020000FAF7B6FF05466061FFF7FAF80146F08895
:100210007F1EC019FAF7ACFF02228542606801D147
:10022000104300E090436060E1681040084303D051
:10023000002000F0B9F8F8BD0220FAE7882100207C
:10024000842F002010B502484069FDF77FFF10BDE4
:100250008821002010B5FFF7C1F8441EFFF7D0F841
:100260004443FFF7CDF804494A69521E5043CA6817
:100270002146FDF770FF10BD88210020F8B5104819
:100280001422017851430C182569FFF7B9F801468B
:10029000E088228980184019FAF76AFF0F46FFF7B5
:1002A0009DF8461EFFF7ACF84643E0882289F11915
:1002B0008018044A40191269FDF74DFFF8BD00008F
:1002C000842F00208821002070B5FFF799F805469B
:1002D000FFF784F8441EFFF793F860432946FAF7C6
:1002E00047FFFDF733FF70BD70B5FFF789F886084B
:1002F000FFF786F80749496948430446FFF76EF857
:10030000451EFFF77DF8684332462146FDF723FF7F
:1003100070BD00008821002070B5144814220178B7
:1003200051430C18241DFFF76BF86188104E88426A
:1003300011D2FFF765F861880D1AFFF761F882089E
:10034000A188E0684018216940194919FDF703FFA9
:10035000FFF756F807E0A288E06880188A0821694C
:10036000FDF7F9FE6088F06170BD0000842F002069
:100370008821002010B505480079000703D401202A
:1003800000F012F810BD00F003F810BD8821002025
:1003900010B504480822416891434160407800F05C
:1003A00003F810BD882100200249487002498000EE
:1003B0000858004788210020740C020010B504463C
:1003C000FFF708F92046FCF707FE10BD10B50548F9
:1003D0000079000702D4FDF7EDFA10BDFFF7D8FF52
:1003E00010BD00008821002010B500F0C1F810BD3C
:1003F00070B5154800210160012382051360026871
:10040000002AFCD0114DA8694360C3600522120286
:1004100084186160C21DF932116451649164D16421
:10042000012203261204360286197260D21113507B
:10043000042222616A6B2264FF2205326264036037
:100440000020296170BD0000000100400C21002047
:10045000FEB51F4C00252769E06802906846FDF74D
:10046000F1FD0190FEF71EF806460198002822D003
:1004700000230098E16817E00E680A46864202D918
:10048000301A086012E0801BF31800261660D66848
:10049000D169B446002E07D0FE183602360A5660DF
:1004A00066469660D56115460029E5D12846E1608B
:1004B000FEF756F806E02846FEF752F8002801D16C
:1004C000002E02D00298FDF7F7FA00202071FEBD41
:1004D000D821002001200249000508607047000073
:1004E00000E200E010B50E4BD968002906D0026882
:1004F0000C68A24204D8A21A0A60C161D86010BD7B
:100500000B4604E00B46C969121B002904D00C6895
:100510009442F7D3A41A0C600260C161D86110BD87
:10052000D821002070B50024104A234625461E011C
:100530009659864205D118018018C5608160D8B2ED
:1005400070BD5B1C202BF2DB00231E019659002E90
:1005500004D05B1C202BF8DB204670BD1C01105121
:10056000A0180371C560DCB28160F5E7643100203A
:1005700070B50024094D264621016858002809D08D
:100580004819C268521CC26083689A4202DBC66086
:1005900068588047641C202CEEDB70BD643100205D
:1005A000F8B51D4DEC68002C34D01C48002740687D
:1005B0002969401A0602360A2068B04218D8361A4D
:1005C000C7192246107CE46900280FD0002010745F
:1005D0006B69002B07D0916950699847002805D0B6
:1005E000FCF7C8F902E0516990698847002CE3D113
:1005F0006978A878814206D1401CC0B2A870022850
:1006000001D10020A87004490006800D18310F5058
:10061000FFF760FFF8BD0000D82100200015014061
:100620000278002804D0202A05D90120C043704751
:100630000020C04370471301044A0021D1509A188A
:100640009160D160FF21017000207047643100206B
:10065000FF2107481D31002242500648828A8168E6
:10066000895C828A521C82820348C1617047000003
:1006700000200040682F00200025004070B505468E
:10068000244892B00FC809AC0FC41C2102A8FAF785
:10069000B2FD6946087A0C210843694608720024B5
:1006A0000394059406940794294609A8089463DFE7
:1006B00000282DD129786846817117498180012051
:1006C00001466846103100940170012001466846D9
:1006D000103141708278F9200240F720921C0240CC
:1006E000EF200240012632436846827014210DA893
:1006F000FAF781FD01A80D9068460E908687C487A1
:10070000142110A8018068882B1D0DAA02A9A2DF60
:1007100012B070BD140C0200F53600001FB50021A8
:100720006A4611701072044882680192817506C889
:10073000684690471FBD0000682F002010B5017863
:10074000022901D0012902D14068FCF713F910BD3C
:100750007CB50178284D01290AD002292FD0002923
:100760002CD129462548FCF711F9002833D036E072
:100770004068017821481038FCF725F91F4C103CDF
:10078000002805D001216A4611700190684608E0F2
:10079000A068E168081A012805D1002069460870A0
:1007A000684669688847A068E168081AA188884295
:1007B00004D811480121401CFEF7DEFA7CBD02215D
:1007C0006A461170C06801900B480121401CFEF779
:1007D000D3FA68460CE001210748FEF74DFB0748B5
:1007E0008168C0688842E9D103206946087068467C
:1007F000696888477CBD000080210020102F002000
:10080000F0B5454D012185B049022846FEF744FC6C
:1008100001270026414C002824D0FF2125312846FD
:10082000FEF735FC00281DD0FF2025302E508120FA
:100830003B4980008860A07E002800D16F600221C3
:10084000684601703749086808600390E17D684692
:100850000172E0680190E675267606CC6846083C91
:1008600090472BE004212846FEF716FC002825D0EF
:10087000FF2109312846FEF70AFC00281ED0FFF7A9
:100880009BF8E07D617E884218D1207E002808D048
:10089000627EE168E0752069E06026766676104643
:1008A0000AE0A07E002800D16F6081201C498000F2
:1008B0008860E675607EE168FFF7F4F8FF211D317E
:1008C0002846FEF7E4FB00280DD0A18AA07D8142D6
:1008D00002D2FFF7BDFE06E0FF211D316E50002859
:1008E00001D0FFF71BFFFF2145312846FEF7CFFB64
:1008F00000280ED0FF2045302E50A07E002800D0CA
:100900002F60E07D002804D0E675607EE168FFF787
:10091000C9F805B0F0BD000000200040682F00209D
:1009200000230040802400400870000A4870022024
:100930007047000038B51549154A488890420FD0D5
:100940004A78144C521CD2B24A70237B934208D38B
:10095000091D75DF002803D0A169002900D0884750
:1009600038BD00254D70217C002907D03B2176DF62
:10097000002803D0A169002900D0884761690029B7
:10098000EED068460570884738BD00006C21002015
:10099000FFFF0000E42E002001200C4B01290DD0A8
:1009A000022907D003290DD0042902D1002A00D141
:1009B00058707047002AFCD198707047002AFCD10B
:1009C00018707047002AFCD1D8707047D4200020DE
:1009D000EFF30580C005C00D1AD0103840B20028D2
:1009E00008DA0107090F083989080C4A89008918B3
:1009F000C96904E081080A4A8900891809688007E2
:100A0000C00EC1400806800F012803D0032803D080
:100A100002207047002070470120704700ED00E081
:100A200000E400E042788378521CD2B2934200D1B5
:100A300000220378934201D1002070470A70416878
:100A400040781822504308187047FFB583B0164607
:100A50000C9D0D9C1F46022200950194039800F006
:100A60000CF8002807D13B4610223146009501942E
:100A7000039800F002F807B0F0BDFFB583B0074659
:100A800000200C9C8646268805463AE07868A90036
:100A900042181188684681805188C18000226946C9
:100AA00001A865DF002839D16846017805988142A0
:100AB00026D17046002801D0002200E002222088C2
:100AC000891842180D998A4227D8714600290AD1FF
:100AD000401C80B22080069A049911542088401C42
:100AE000208001208646218806980A18694601A8B8
:100AF00065DF002812D169462088097840182080D7
:100B00006D1C3888A842C1DC704600280AD02088B5
:100B1000801B401E80B2FF2802D90C2007B0F0BD18
:100B2000069988550020F9E710B502480078FEF7CD
:100B300019FA10BD0921002010B57D2109010248D4
:100B4000FFF7F0FC10BD0000290B02000EB50C49A8
:100B50000868896800900B48029101900A4968462C
:100B6000FEF71AFA002801D0FBF704FF0748FEF74A
:100B7000D7F9002801D0FBF7FDFEFEF7FDF90EBD09
:100B8000CC0B020088130000910B02000921002009
:100B900070470179002902D1007B002800D0012094
:100BA00070470000082400200100000700400040BA
:100BB000000400000300000002000000010000002B
:100BC000FF00000000000000AA5503000100000023
:100BD000D007000001000000FFC1FBE84C90728BC1
:100BE000E7B3518963AB232302841872AA612F3BB8
:100BF00051A8E53749FBC9CA0C18532CFD00000069
:100C0000C42E0020FB349B5F800000800010000099
:100C1000FEE70000FB349B5F8000008000100000B6
:100C2000FEE70000FB349B5F8000008000100000A6
:100C3000FEE70000090000000B0000000A000000B1
:100C400008000000000000000000000000E0D701E4
:100C500003000000090000000B0000000A00000073
:100C600008000000000000000000000000E0D701C4
:100C700003000000C9020200E9020200450202006E
:100C80007D0202005502020075030200ADDC010086
:100C900059DC0100CD0302004DE201000300000019
:100CA0000200000001000000FF0000000000000042
:100CB000AA55030001000000D00700000100000059
:100CC000080910110000000000E0D701EC0C020040
:100CD000802000208803000096B70100500F02001A
:100CE00008240020A01B0000DEBC010023FFFF50F1
:100CF00008FFFF4001E7FE0123703E180CE4E247C5
:100D00006BA75A01600101101C0910014A402B1108
:100D1000363133646F674724F15012345659190144
:100D200023E3048042111C0808014303100303124B
:100D300080AA401427294176715B06145555550346
:100D400012710229D401AE00FF00891112239B32D7
:100D50002446AD573665BF74488CC19D5AAFD3BE8B
:100D60006CCAE5DB7EE9F7F88110080193331A229B
:100D7000A5562C47B7753E64C99C408DDBBF52AE6B
:100D8000EDDA64CBFFF976E802218B30100299137B
:100D90002667AF763444BD554AADC3BC588ED19F4B
:100DA0006EEBE7FA7CC8F5D983310A20911218035B
:100DB000A7772E66B5543C45CBBD42ACD99E508F2B
:100DC000EFFB66EAFDD874C904428D5316619F702B
:100DD0002004A9153227BB364CCEC5DF5EEDD7FC0B
:100DE0006888E1997AABF3BA85520C4397711E601B
:100DF000A1142805B3373A26CDDE44CFDFFD56ECEB
:100E0000E9986089FBBB72AA06638F7214409D51FA
:100E10002225AB343006B9174EEFC7FE5CCCD5DDCA
:100E20006AA9E3B8788AF19B87730E6295501C41DA
:100E3000A3352A24B1163807CFFF46EEDDDC54CDAA
:100E4000EBB962A8F99A708B1023088481951AA7D0
:100E500093B62CC2A5D33EE1B7F04008C919522B76
:100E6000DB3A644EED5F766DFF7C899410DE859BE6
:100E7000B712A6ADD224C3BFF136E0C1184809D3DA
:100E80003B5A2AE55E6C4FF77D7E6C0AA583B41849
:100E90008691972EE3A7F23CC0B5D14229CB3850BA
:100EA0000AD91B666FEF7E744CFD5D8BB502A49969
:100EB000961087AFF326E2BDD034C1C3394A28D19A
:100EC0001A580BE77F6E6EF55C7C4D0CC685D71EFD
:100ED000E597F42880A1913AA3B3B2444ACD5B567A
:100EE00069DF78600CE91D722FFB3E8DD604C79F29
:100EF000F516E4A9902081BBB332A2C55A4C4BD75A
:100F0000795E68E11C680DF33F7A2E0EE787F61CC8
:100F1000C495D52AA1A3B03882B193466BCF7A5439
:100F200048DD59622DEB3C700EF91F8FF706E69DE8
:100F3000D414C5ABB122A0B9923083C77B4E6AD519
:100F4000585C49E33D6A2CF11E780F1324F400002D
:040000050001B0C185
:00000001FF
